:100000003CEF03F00000000000EF00F000000000F3
:0A0010000000000000000000F3D71C
:0E001C0072B202D00000FCD767C073FF120062
:0E002A00ACB202D00000FCD767C0ADFF1200E0
:10003800F250026EF29E0500FF6A0150FE6E0050FB
:08004800FD6E02BEF28E1200F3
:10005000026AC7B408D01F0EC514016E0150000A11
:0C00600002E1FF0E026E02C000F0120070
:10006C0033C063F034C064F035C065F036C066F060
:10007C000001616B626BE6DF0050000A01E00AD000
:10008C0000016251120A02E18E0E611903E0614B0C
:10009C00622BF1D70001120E625D02E18F0E615DE1
:1000AC0003E37B0E606F34D0C580C5A030D0000E4A
:1000BC00006E361808E10050351805E10050341870
:1000CC0002E13350000A22E0000E006E661908E1CE
:1000DC000050651905E10050641902E16351000AF2
:1000EC000FE139C0E1FF3AC0E2FF050EE66E37C002
:1000FC0000F038C001F09ADF010E0001606F08D0EB
:10010C00010E635F000E645B655B665BCED7606B54
:06011C0060C000F01200BB
:04012600C58412007A
:10012A0033C062F034C063F035C064F036C065F0A5
:10013A009E9660C0C9FFC7A431D0000E006E361863
:10014A0008E10050351805E10050341802E1335037
:10015A00000A23E0000E006E0001651908E1005054
:10016A00641905E10050631902E16251000A0FE1C6
:10017A0039C0E1FF3AC0E2FF040EE66E37C000F074
:10018A0038C001F054DF010E0001616F4BD0010E3F
:10019A00625F000E635B645B655BCDD733C062F060
:1001AA0034C063F035C064F036C065F09EB631D015
:1001BA00000E006E361808E10050351805E10050AF
:1001CA00341802E13350000A23E00001000E006EE9
:1001DA00651908E10050641905E10050631902E14C
:1001EA006251000A0FE139C0E1FF3AC0E2FF040E92
:1001FA00E66E37C000F038C001F019DF010E0001C9
:10020A00616F10D0010E625F000E635B645B655B19
:10021A00CDD7C5BC03D00001616B04D00001C584F1
:0A022A00020E616F61C000F01200C7
:1002380019DF780E606F75DF606B73DF5FC060F089
:0602480070DF6DDF120003
:1002580009DF780E606F65DF400E606F62DF5DC09A
:0802680060F05FDF5CDF1200B3
:10027A005E50B00F5F6EDBDF0F0E5D145F6ED7DF6F
:10028A00F00E5D145F6E5F325F9E5F325F9E5F327B
:0E029A005F9E5F325F9E100E5F26C9DF12006E
:1002AE000D0E0001676FBADE0A0E0001676FB6DE33
:0202BE0012002C
:1002C4005B6A59C0E9FF5AC0EAFFEECF5CF05C50AC
:1002D400000A0DE05CC067F0A6DE5B2A5B5059247F
:1002E400E96E000E5A20EA6EEECF5CF0F0D71200F1
:1002F6002A0E536E000E546E670E556E000E566E25
:10030600FF0E3F6EFF0E406E000E416E000E426EF7
:10031600FF0E436EFF0E446E000E456E000E466ED7
:10032600FF0E476EFF0E486E000E496E000E4A6EB7
:10033600AC8A900EAB6E948E949C9EAA03D0AECFE0
:0603460000F0FBD71200DD
:10034C00336A346A356A366A500E156E000E166EB4
:10035C00000E176E000E186E6C0E196E000E1A6ED3
:10036C00000E1B6E000E1C6EFF0E1D6EFF0E1E6E21
:10037C00000E1F6E000E206EFF0E3B6EFF0E3C6ECD
:10038C00FF0E3D6EFF0E3E6E2A0E4B6E010E4C6E36
:10039C00600E4D6E000E4E6E260E4F6E010E506EA0
:1003AC00000E516E000E526E949894968B988B960C
:0E03BC0094889486C79EC79C380EC66E1200A9
:1003CA00200E5F6E34DF5F6A32DF210E5F6E2FDF31
:1003DA0059C05FF02CDF5950070F5F6E28DF220EDD
:1003EA005F6E25DF5AC05FF022DF5A50010F5F6E41
:1003FA001EDF5B6A5C6A4E0E5B24F66E020E5C20A0
:10040A00F76E000EF86E000E5CBEFF0EF822F6CFF5
:10041A00F6FFF7CFF7FFF8CFF8FF0900F5CF5DF049
:10042A0016DF000E5C1802E1070E5B1803E05B4A58
:10043A005C2AE1D7200E5F6EFADE5F6AF8DE210ED3
:10044A005F6EF5DE5F6AF3DE7F0E5F6EF0DE220E10
:06045A005F6EEDDE1200F2
:10047E00210E5F6EDADE5F6AD8DE7F0E5F6ED5DE2E
:10048E00220E5F6ED2DE5F6AD0DE030E5F6ECDDEB1
:10049E00D30E5F6ECADE400E5F6EC7DE5D6A5E6AA9
:1004AE00E5DE596A5950B00F5F6EBFDE010E5F6E0A
:1004BE00BCDE100E5F6EB9DE0D0E0D6E0D2EFED76C
:1004CE005A6A5D6AC2DE0D0E0D6E0D2EFED75A50A3
:1004DE00800A02E05A2AF5D75950040A02E0592A36
:1004EE00E1D72E0E5F6EA1DE5D6A5E6ABFDE120080
:10051C00AE0E5F6E8BDE050E0B6E0F0E0C6EF10EBB
:10052C000D6E0D2EFED70C2EFCD70B2EFAD7AF0E60
:10053C005F6E7CDE030E0B6E080E0C6E770E0D6E6E
:10054C000D2EFED70C2EFCD70B2EFAD7B00E5F6EED
:10055C006DDE5F6A6BDE030E5F6E68DE200E5F6E13
:10056C0065DE020E5F6E62DE210E5F6E5FDE5F6A1D
:10057C005DDE7F0E5F6E5ADE220E5F6E57DE5F6AA7
:10058C0055DE030E5F6E52DEA10E5F6E4FDEA40EC3
:10059C005F6E4CDEA60E5F6E49DEC80E5F6E46DEE9
:1005AC00D30E5F6E43DE3F0E5F6E40DED50E5F6E88
:1005BC003DDE800E5F6E3ADEA80E5F6E37DE3F0EBC
:1005CC005F6E34DED60E5F6E31DE800E5F6E2EDE19
:1005DC00D90E5F6E2BDE1F0E5F6E28DEDA0E5F6E9D
:1005EC0025DE200E5F6E22DEEE0E5F6E1FDE810EAC
:1005FC005F6E1CDE7F0E5F6E19DE2E0E5F6E16DEDA
:10060C00DB0E5F6E13DE400E5F6E10DE8D0E5F6EC6
:10061C000DDE140E5F6E0ADEAF0E5F6E07DE12008B
:10067800D390D392D388D38AD38C9B9C150E0B6EC0
:100688004B0E0C6EBE0E0D6E0D2EFED70C2EFCD72B
:100698000B2EFAD70000826A8B6A0F013A6B800E24
:1006A800946E386B806A9298576A586A89880B0EDC
:1006B8000B6E260E0C6E5D0E0D6E0D2EFED70C2EDB
:1006C800FCD70B2EFAD70000000089980B0E0B6E92
:1006D800260E0C6E5D0E0D6E0D2EFED70C2EFCD761
:1006E8000B2EFAD700000000000E581802E1040E85
:1006F800571803E0574A582AD9D7B886B06ACF0E98
:10070800AF6EAC84F4DD540E216E650E226E730E4E
:10071800236E740E246E200E256E4F0E266E4C0E20
:10072800276E450E286E440E296E200E2A6E530E33
:100738002B6E530E2C6E440E2D6E310E2E6E330E14
:100748002F6E300E306E360E316E326A210E596EB3
:10075800000E5A6EB3DDA7DD280EC86EF3DD150E48
:100768000B6E4B0E0C6EBE0E0D6E0D2EFED70C2EA4
:10077800FCD70B2EFAD70000CDDE7DDE0A0E596EAF
:100788000A0E5A6E1EDE290E0B6E960E0C6E7F0E2A
:100798000D6E0D2EFED70C2EFCD70B2EFAD7FFD7D9
:08024E000F080F00F8888888F2
:020000040030CA
:0D000100A81F3CFFBF81FF0FC00FE00F40A4
:00000001FF
